:020000020000FC
:0200000019C025
:02000A0055C1DE
:100034000FED0DBF8D9AB89AC09809D01BD011D07E
:100044002CD07894EEEFF2E050D01ED1FECF899AF6
:1000540008E00AB906E003B900E002B909E109B908
:10006400089503E300BF09E003BF0FE306BF00E206
:100074000CBF089502E0006C0FBD09E10EBD09B785
:10008400006809BF10E01BBD00E80ABD15BD0FEFF5
:1000940004BD6627772788270895442755270895A0
:1000A400EF93FF931F931FB7E0E6F0E0E40F0083A4
:1000B40043954F711FBF1F91FF91EF9108950F93C7
:1000C4001F93EF93FF931FB7451749F05D9B07C03C
:1000D400E0E6F0E0E50F008153955F710CB91FBFB6
:1000E400FF91EF911F910F9108950F931F931FB7E5
:1000F4000591002311F0D4DFFBCF1FBF1F910F9197
:1001040008950F931F931FB70F700A3018F00A5009
:10011400016401C00063C4DF1FBF1F910F910895E4
:100124000F931F932F932FB72F930091A00010913B
:10013400A10020E00130120710F4C09A07C001505A
:10014400120B0093A0001093A100C0982F912FBF11
:100154002F911F910F910895EF93FF931F931FB752
:10016400E0E8F0E0E60F008363956F711FBF1F9115
:10017400FF91EF9108951F93EF93FF931FB7E0E86A
:10018400F0E0E70F7617F1F3008173957F711FBFDD
:10019400FF91EF911F9108951F931FB7ECDFC02EBD
:1001A400EADFD02E0C2DCD1409F001C002E01FBFF0
:1001B4001F9108951F932F933F933FB7BB24AA2405
:1001C40011E024E0E9DF023011F401E008C0BB0CC7
:1001D400002311F0B12AA1262A95A1F700E03FBF20
:1001E4003F912F911F9108951F932F932FB711E0E3
:1001F400D3DF023011F401E006C0002319F0A12678
:10020400AA20C9F700E02FBF2F911F9108951F93D3
:100214002F933F93EF93FF933FB711271093AD00B4
:100224001AE0E2EAF3EAC6DF002339F5DDDF002352
:1002340021F5B1922091AD002B252093AD001A95A4
:1002440091F7B8DF0023C9F42091AD002B2520934A
:10025400AD00222389F4E2EAF3EA1AE0019151DFC6
:100264001A95E1F70DE01CDF04EF0093A00001E014
:100274000093A10000E001C001E03FBFFF91EF91B6
:100284003F912F911F91089501E0602E74DF07952F
:10029400771C881C991C03E090220AEA70168006D9
:1002A40002E0900621F4B3DF772488249924EECF6A
:1002B40008950F931F932F931FB72227829921E04C
:1002C4002F1511F493950AC00F2D9C3008F044DFCC
:1002D4000F2D943018F040DF91E0F22E8395883092
:1002E40009F4EDDE8C3009F41BDF803109F4882732
:1002F4001FBF2F911F910F9118955265616465720C
:0C030400206765737461727465740D00ED
:00000001FF
